:100000000128831686138610061386128312861320
:1000100086109901960114308C0000308D000C0878
:100020009A000D089B00051C252806178612160845
:100030008C0001300C0203010318FF3E0319252830
:1000400016088C0001300C029600851C3328861699
:1000500006131608643C03010318FF3E03193328F6
:100060001608013E9600051D642801308C00190811
:100070000C0299001908031D861703198613051D24
:10008000642864308C0000308D000C0897000D0847
:10009000980017088C0018088D0000308E00003082
:1000A0008F00CC200319632817088C0018088D00D6
:1000B00001308C02031C8D0300308D020C08970068
:1000C0000D08980049283F288519672864281608D4
:1000D0008C008D0102308E0000308F00B3200C08A0
:1000E00097000D08980017088C0018088D00003044
:1000F0008E0000308F00CC2003198D2817088C004B
:1001000018088D0001308C02031C8D0300308D0215
:100110000C0897000D089800732886141E308C0078
:1001200000308D000C0897000D08980017088C000F
:1001300018088D0000308E0000308F00CC2003198D
:10014000B02817088C0018088D0001308C02031CA1
:100150008D0300308D020C0897000D08980096283A
:100160008610132801289001910103108D0C8C0C2E
:10017000031CC1280E0890070318910A0F08910765
:1001800003108E0D8F0D0C080D04031DB5281008EB
:100190008C0011088D0008000D080F02031DD228E5
:1001A0000C080E02031CD7288C018D010800FF38B3
:0601B0008C008D00080028
:02400E00F93F78
:00000001FF
